S024000062696E2F6F70656E626C745F6F6C696D65785F73746D3332703130332E737265639B
S3150800000058110020A94800088D4800088D480008A6
S315080000108D4800088D4800088D4800088D4800085E
S315080000208D4800088D4800088D4800088D4800084E
S315080000308D4800088D4800088D4800088D4800083E
S315080000408D4800088D4800088D4800088D4800082E
S315080000508D4800088D4800088D4800088D4800081E
S315080000608D4800088D4800088D4800088D4800080E
S315080000708D4800088D4800088D4800088D480008FE
S315080000808D4800088D4800088D4800088D480008EE
S315080000908D4800088D4800088D4800088D480008DE
S315080000A08D4800088D4800088D4800088D480008CE
S315080000B08D4800088D4800088D4800088D480008BE
S315080000C08D4800088D4800088D4800088D480008AE
S315080000D08D4800088D4800088D4800088D4800089E
S315080000E08D4800088D4800088D4800088D4800088E
S315080000F08D4800088D4800088D4800088D4800087E
S315080001008D4800088D4800088D4800088D4800086D
S315080001108D4800088D4800088D4800088D4800085D
S315080001208D4800088D4800088D4800088D4800084D
S315080001308D4800088D4800088D4800088D4800083D
S315080001408D4800088D4800088D4800088D4800082D
S3150800015000B5C7B0684600214FF48C7204F0D6FB90
S3150800016044F6AC10C0F60000694602F0B1FD48B985
S31508000170009B002043B19DF8080080F01000C0F3F2
S31508000180001001E00020FFE747B05DF804FB00BF60
S3150800019044F6AC10C0F60000704700BF08B540F240
S315080001A00800C2F20000002380F8283244F6CC1179
S315080001B0C0F600010A2202F0F7F930B940F2080346
S315080001C0C2F20003012283F8282208BD70B540F266
S315080001D00803C2F2000393F82832012B05D140F236
S315080001E00800C2F2000002F0A9FC04F0BBF800F116
S315080001F064064FF48844C4F20004402503E004F082
S31508000200B1F8864205D32046294600F083FE002829
S31508000210F5D044F6AC10C0F6000002F083FD70BDC0
S3150800022008B540F20803C2F2000393F82832012BFE
S3150800023005D140F20800C2F2000002F07FFC08BDBA
S3150800024070B5064640F20803C2F2000393F8283256
S31508000250012B10D140F20801C2F2000102F0EEFDB6
S31508000260002808DA40F20800C2F20000002380F8ED
S31508000270283202F063FC317889B14FF48844C4F21D
S3150800028000048025204600F041FE2046294600F05D
S3150800029041FE0028F9D016F8011F0029F2D170BDD9
S315080002A000B583B00023009301934FF48053C4F242
S315080002B002031A6842F001021A6059680022CFF652
S315080002C0FF020A405A601A6822F0847222F48032C9
S315080002D01A601A6822F480221A605A6822F4FE020A
S315080002E05A604FF41F029A601A6842F480321A6004
S315080002F04FF48053C4F2020340F2DC52196801F449
S3150800030000310191009901310091019911B90099C3
S315080003109142F3D14FF48053C4F202031B6813F4DD
S31508000320003F06D144F6DC10C0F600006E2103F04B
S3150800033061FD4FF40053C4F202031A6842F010023A
S315080003401A601A6822F003021A601A6842F002025A
S315080003501A604FF48053C4F202035A685A605A6806
S3150800036042F400525A605A6842F480625A605A68E7
S3150800037022F47C125A605A6842F4E8125A601A68E3
S3150800038042F080721A604FF48053C4F202031A686E
S3150800039012F0007FFBD04FF48053C4F202035A6870
S315080003A022F003025A605A6842F002025A604FF479
S315080003B08053C4F202035A6802F00C02082AFAD1E2
S315080003C04FF48053C4F202039A6942F009029A6113
S315080003D04FF44062C4F20102516821F00F015160E6
S315080003E0516841F008015160516821F0F0015160EF
S315080003F0516841F0B00151600022C4F2010251680F
S3150800040021F4C0415160516841F480415160DA6974
S3150800041042F00072DA61DA6942F40032DA619A6906
S3150800042042F005029A614FF40063C4F201031A68A8
S3150800043022F470621A601A6842F430621A601A6806
S3150800044022F470421A601A6842F480421A6002F076
S3150800045099FD02F0A7FDFCE738B501464FF4605058
S31508000460C4F2000000F038FD4FF46054C4F20004F2
S3150800047001252046294600F043FD0028F9D04FF40F
S315080004806050C4F2000000F029FDC0B238BD00BFBC
S3150800049070B503F067FF00F5FA76FF252846FFF7E3
S315080004A0DBFF0446FF2803D003F05CFF8642F5D83D
S315080004B0FF2C14BF0020012070BD00BF08B54FF403
S315080004C04060C4F201004FF4805100F0ADFCFF20FB
S315080004D0FFF7C2FF08BD00BF10B54FF44060C4F275
S315080004E001004FF4805100F0A1FCFF20FFF7B4FF94
S315080004F0FFF7CEFF044610B9FFF7E0FF00E001243E
S31508000500204610BD38B504460D4610F0800F07D0BA
S3150800051037200021FFF7F6FF01283AD804F07F04B8
S31508000520FFF7CCFFFFF7D8FF48B344F04000FFF7CA
S3150800053093FF280EFFF790FFC5F30740FFF78CFFE0
S31508000540C5F30720FFF788FFE8B2FFF785FFE4B198
S31508000550082C16D00120FFF77FFF0C2C02D1FF20B4
S31508000560FFF77AFF0A24FF252846FFF775FF10F0E4
S31508000570800F0ED0631E13F0FF04F5D138BDFF209F
S3150800058038BD8720FFF768FFECE79520FFF764FF83
S31508000590E8E738BD38B505460C46FFF779FF034648
S315080005A020B32046FFF758FFFD2C08BF01231DD0B6
S315080005B0AC1C05F2022514F8020CFFF74DFF14F8DF
S315080005C0010CFFF749FF0234AC42F4D1FF20FFF7D4
S315080005D043FFFF20FFF740FFFF20FFF73DFF00F036
S315080005E01F00052814BF00230123FFE7184638BD5E
S315080005F0F8B504460D4603F0B5FE00F16407FF267C
S315080006003046FFF729FFFF2804D103F0ABFE8742E7
S31508000610F6D818E0FE2818D10234FF263046FFF730
S315080006201BFF04F8020C3046FFF716FF04F8010C0E
S315080006300234023DF2D1FF20FFF70EFFFF20FFF73D
S315080006400BFF0120F8BD0020F8BD0020F8BD00BF53
S315080006502DE9F04389B0002840F0848140F2000378
S31508000660C2F200031B7813F0020F06D040F2000313
S31508000670C2F200031878C0B27FE10820012100F019
S31508000680D7FB4FF48040012100F0E4FB4FF480587B
S31508000690ADF800804FF010098DF8039003278DF808
S315080006A002704FF44064C4F201042046694600F023
S315080006B069FB2046414600F0B7FB4FF42043ADF8EE
S315080006C000308DF8027018238DF8033020466946ED
S315080006D000F058FB4FF48046ADF8006048238DF8CB
S315080006E003302046694600F04DFB0025ADF808505A
S315080006F04FF48273ADF80A30ADF80C50ADF80E50D1
S31508000700ADF810504FF40073ADF812303823ADF839
S315080007101430ADF816500723ADF8183006FA09F06C
S3150800072040F4605002A900F0A7FB06FA09F040F46D
S315080007306050294600F0D6FB06FA09F040F46050EE
S31508000740012100F0BBFB2046414600F06DFB4FF44B
S315080007500045ADF804508DF806708DF807902046D0
S3150800076001A900F00FFB2046294600F05DFB0A2789
S315080007704FF46054C4F2000402264FF0FF08012526
S315080007802046314600F0BCFB0028F9D020464146F9
S3150800079000F0A2FB2046294600F0B2FB0028F9D05B
S315080007A0013FEDD14FF40043ADF8043003238DF833
S315080007B0063018238DF807304FF44064C4F201045C
S315080007C0204601A900F0DEFA20464FF4805100F0D9
S315080007D02DFB00200146FFF795FE012840F0C48056
S315080007E003F0C0FD00F57A7408204FF4D571FFF7C1
S315080007F089FE012849D10DF11F060DF11B05FF27BA
S315080008003846FFF729FE05F8010FB542F8D19DF8DD
S315080008101E30012B40F0A8809DF81F30AA2B40F00F
S31508000820A380A9274FF0804503F09CFD844205D993
S3150800083038462946FFF766FE0028F5D103F092FDF3
S31508000840844240F291803A200021FFF75BFE00289F
S3150800085040F08A800DF11B04FF252846FFF7FCFDB2
S3150800086004F8010FB442F8D19DF81C2002F04002AA
S31508000870D2B2002A14BF0C22042240F23423C2F258
S3150800088000031A60FFF71AFE27E0A9200021FFF7E8
S3150800089039FE012899BF0227A92501273D460026CA
S315080008A003F060FD844205D928463146FFF72AFE43
S315080008B00028F5D103F056FD844255D910204FF48F
S315080008C00071FFF71FFE00284ED140F23423C2F212
S315080008D000031F60FFF7F2FDAFB340F20003C2F258
S315080008E000031A7802F0FE021A704FF46055C4F23B
S315080008F000052846002100F0E1FA0024ADF808407A
S315080009004FF48273ADF80A30ADF80C40ADF80E40DE
S31508000910ADF810404FF40073ADF812300823ADF867
S315080009201430ADF816400723ADF81830284602A94A
S3150800093000F0A2FA2846214600F0D4FA28460121FA
S3150800094000F0BCFA07E040F20003C2F200031A788E
S3150800095042F001021A7040F20003C2F2000318784E
S31508000960C0B20AE0012008E040F23423C2F20003D4
S3150800097000221A60FFF7A2FDE5E709B0BDE8F0839B
S3150800098030B940F20003C2F200031878C0B27047CB
S315080009900120704770B50D461C46D3F1010338BFD8
S315080009A0002300280CBF184643F0010000283BD15D
S315080009B040F20003C2F200031B7813F0010F35D191
S315080009C040F23423C2F200031B6813F0080F08BF75
S315080009D05202012C0ED111201146FFF793FDE8B9FA
S315080009E028464FF40071FFF703FED0F1010438BF23
S315080009F0002413E012201146FFF784FD70B94FF466
S31508000A00007628463146FFF7F3FD18B105F500755F
S31508000A10013CF6D10C200021FFF774FDFFF74EFDCF
S31508000A20201C18BF012070BD042070BD032070BDB6
S31508000A30F8B50E4617461D46D3F1010338BF002305
S31508000A4000280CBF184643F0010000284BD140F29D
S31508000A500003C2F200031B7813F0010F45D140F2E0
S31508000A600003C2F200031B7813F0040F3FD140F2D3
S31508000A703423C2F200031B6813F0080F08BF57029D
S31508000A80012D0DD118203946FFF73CFD28BB30460D
S31508000A90FE21FFF77FFDD0F1010538BF00251CE0D8
S31508000AA013F0060F03D097202946FFF72BFD1920D0
S31508000AB03946FFF727FD80B9FC2430462146FFF763
S31508000AC069FD18B106F50076013DF6D10020FD2135
S31508000AD0FFF760FD002808BF0125FFF7EFFC281C7B
S31508000AE018BF0120F8BD0420F8BD0320F8BD022078
S31508000AF0F8BD00BF70B584B01446002840F03D81AB
S31508000B0040F20003C2F200031B7813F0010F18BF6E
S31508000B10032040F034810E2900F21481DFE811F039
S31508000B200F00160012015C001201120112011201D7
S31508000B3012011201C200CA00D900E800F700FFF747
S31508000B40CBFCD0F1010438BF002412E109200021B2
S31508000B50FFF7D8FC002840F0F78068461021FFF719
S31508000B6047FD002800F0F2809DF800309B09012B14
S31508000B7010D19DF8072002F03F02120401329DF8B9
S31508000B8009309DF8081003EB012313449B022360E8
S31508000B900024EEE09DF808209DF807309B0003EB43
S31508000BA092139DF8062002F0030203EB822201321B
S31508000BB09DF8053003F00F039DF80A1003EBD113D7
S31508000BC09DF8091001F0030103EB4103073B02FA04
S31508000BD003F323600024CCE040F23423C2F200037E
S31508000BE01B6813F0040F22D08D200021FFF78AFC22
S31508000BF0002840F0AD80FF20FFF72EFC6846102144
S31508000C00FFF7F6FC002800F0A5803025FF263046C1
S31508000C10FFF722FC6B1E13F0FF05F8D19DF80A308A
S31508000C201B09102202FA03F323600024A1E009201D
S31508000C300021FFF767FC002840F08E8068461021E7
S31508000C40FFF7D6FC002800F0898040F23423C2F270
S31508000C5000031B6813F0020F12D09DF80A2002F059
S31508000C603F029DF80B30DB0903EB420201329DF887
S31508000C700D309B09013B02FA03F32360002478E058
S31508000C809DF80B309DF80A20C2F38402013203F066
S31508000C9003015B0903EBC103013303FB02F3236082
S31508000CA0002466E040F23423C2F200031B68137086
S31508000CB000245EE009200021FFF724FC00284FD11C
S31508000CC020461021FFF794FCD0F1010438BF002418
S31508000CD04FE00A200021FFF715FC002842D12046E4
S31508000CE01021FFF785FCD0F1010438BF002440E04D
S31508000CF03A200021FFF706FCB0BB0025FF26304648
S31508000D00FFF7AAFB60550135042DF8D12EE040F215
S31508000D103423C2F200031B6813F0040F08BF012432
S31508000D2027D08D200021FFF7EDFB08BBFF20FFF73A
S31508000D3093FB20464021FFF75BFCD0F1010438BF46
S31508000D40002416E0042414E0012412E0012410E033
S31508000D5001240EE001240CE001240AE0012408E045
S31508000D60012406E0012404E0012402E0002400E056
S31508000D700124FFF7A3FB204601E00420FFE704B0A7
S31508000D8070BD00BF2DE9F001CB7803F00F0513F015
S31508000D90100F1CBF8B781D430B78F3B1076800232F
S31508000DA001264FF00F0C06FA03F20C881440944201
S31508000DB00FD19A000CFA02F827EA080705FA02F298
S31508000DC01743CA78282A08BF446102D0482A08BFB0
S31508000DD004610133082BE6D107600B88FF2B20D965
S31508000DE04768002301264FF00F0C03F1080206FAA4
S31508000DF002F20C88144094420FD19A000CFA02F8B9
S31508000E0027EA080705FA02F21743CA78282A08BF0C
S31508000E104461CA78482A08BF04610133082BE4D123
S31508000E204760BDE8F001704701617047416170474E
S31508000E3039B14FF48053C4F202039A69104398619A
S31508000E4070474FF48053C4F202039A6922EA0000FD
S31508000E509861704739B14FF48053C4F20203DA69D6
S31508000E601043D86170474FF48053C4F20203DA691D
S31508000E7022EA0000D861704710B4028802F4415291
S31508000E804C880B8823438C882343CC8823430C89BE
S31508000E9023434C8923438C892343CC892343134317
S31508000EA09BB20380838B23F400631B041B0C838390
S31508000EB00B8A03825DF8044B704700BF29B103888B
S31508000EC09BB243F0400303807047038823F0400336
S31508000ED01B041B0C0380704781817047808980B290
S31508000EE0704700BF29B103889BB243F400530380BF
S31508000EF07047038823F400531B041B0C03807047B8
S31508000F00038919420CBF002001207047C1F308016C
S31508000F1081807047038819420CBF00200120704762
S31508000F20C278837843EA0222437843EA02220078A9
S31508000F3040EA0220704700BF32B1821811F8013B1F
S31508000F4000F8013B9042F9D1704700BF0239436966
S31508000F50023B99423DBF4289836A02FB0130002069
S31508000F60704700BF00F10B010023DA0142EA530380
S31508000F70DBB210F8012B1344DBB28842F5D11846D0
S31508000F80704700BF30B4046814B325783A2D18BFEB
S31508000F901F2D08D9621C114612F8013B3A2B18BFBF
S31508000FA01F2BF8D801E02B4621463A2B18BF002004
S31508000FB011D1631C994218BF4FF0FF300BD1302D69
S31508000FC018BF4FF0FF3006D102340460002002E05B
S31508000FD04FF0FF30FFE730BC704700BF38B50C460E
S31508000FE0054668B103685BB11A784AB1D988828820
S31508000FF0914205D15878FFF7C3FC10F0010F03D0D2
S3150800100000232360092038BD2B682360002038BDE3
S315080010102DE9F0410446C3780BB3C56A00F13007E1
S31508001020407839462A460123FFF702FDD0B9002346
S31508001030E370236AEA1AA3699A4216D2A678012EA1
S3150800104016D94FF00108A2691544607839462A4630
S315080010504346FFF7EDFC013E012EF4D10BE00020DC
S31508001060BDE8F0810120BDE8F0810020BDE8F081EF
S315080010700020BDE8F0810020BDE8F08170B5044687
S315080010800D46C36A8B4208BF002613D0FFF7C0FF80
S31508001090064678B9607804F130012A460123FFF73D
S315080010A079FC002818BF0126002818BF4FF0FF3525
S315080010B0E562FFE7304670BD10B50446FFF7A8FFA6
S315080010C00346002852D12378032B47D12379012BD5
S315080010D044D104F1300104F50C700B46002203F8E4
S315080010E0012B8342FBD1552384F82E32AA2384F898
S315080010F02F32522384F8303084F83130612384F853
S315080011003230412284F83320722084F8140284F89D
S31508001110150284F8162284F81732236984F81832DF
S315080011201A0A84F819221A0C84F81A221B0E84F853
S315080011301B32E36884F81C321A0A84F81D221A0C3A
S3150800114084F81E221B0E84F81F32E2690132E2621D
S3150800115060780123FFF76CFC002323716078002177
S315080011600A46FFF7C7FC031C18BF0123184610BD23
S315080011702DE9F84305460C461746012998BF02266D
S3150800118040F287804369994228BF022680F0818011
S315080011900378022B45D0032B57D0012B18BF022604
S315080011A077D101EB5108016A01EB5821FFF766FF79
S315080011B0064600286DD108F10109C8F3080814F09D
S315080011C001041FBF05EB080393F8303003F00F0343
S315080011D0FAB21ABF43EA0213DBB2FBB2A84488F894
S315080011E030300123EB70296A284601EB5921FFF7B5
S315080011F045FF064600284CD1C9F3080914B1C7F3C0
S31508001200071708E005EB090393F8303023F00F03BE
S31508001210C7F303271F43A94489F830700123EB70ED
S3150800122037E0016A01EB1421FFF728FF064680BB69
S31508001230630003F4FF73EA1882F83070C7F30727D0
S3150800124082F831700123EB7023E0016A01EBD411B7
S31508001250FFF714FF0646E0B927F07047A40004F428
S31508001260FE7404F13008A8444046FFF759FE00F022
S31508001270704007432C4484F830703B0A88F80130E4
S315080012803B0C88F802303F0E88F803700123EB7098
S31508001290FFE73046BDE8F8838A76C2F30723CB76A4
S315080012A00378032B01BF120C0A75120A4A75704798
S315080012B02DE9F04106460D4600238B758369002B00
S315080012C06ED0436AB3F1FF3F1AD0876A388878B17F
S315080012D00024A046414601F0DBFD58B1FF2C0BD097
S315080012E001342A19507537F8020F0028F2D104E0A4
S315080012F0002402E0002400E000242C440023A37507
S31508001300A87D002423462E275A1CF169CB5C202B86
S3150800131022D0052B08BFE523092A05D108B92919C2
S315080013208F7529194F72013429194B7298B9A3F18F
S315080013304101C9B219290CD8F169097B082A94BF59
S315080013404FF0080E4FF0100E1EEA010F1CBF203397
S31508001350DBB229198B7501340B2A01D01346D3E762
S3150800136038B92B1900229A75F3691B7B934208BF7B
S3150800137014462C4400236372F369DB7A2B72F069F6
S315080013801C30FFF7CDFD2860F3695A7E1B7E43EAC1
S315080013900223AB80F369DA7D9B7D43EA0223EB8067
S315080013A0BDE8F081F8B50C460568012953D96B6983
S315080013B0994252D22B78022B29D0032B3AD0012BF3
S315080013C04DD101EB5106296A284601EB5621FFF754
S315080013D055FE002845D1771CC6F308062E4496F814
S315080013E03060296A284601EB5721FFF747FE002897
S315080013F03AD1C7F308073D4495F8300046EA00207D
S3150800140014F0010F14BF0009C0F30B00F8BD296AD8
S31508001410284601EB1421FFF731FE40BB640004F4B3
S31508001420FF742B1993F830302C4494F8310043EAB2
S315080014300020F8BD296A284601EBD411FFF71EFEE5
S31508001440C0B9A00000F4FE7030302844FFF768FDEC
S3150800145020F07040F8BD0120F8BD0120F8BD01203C
S31508001460F8BD4FF0FF30F8BD4FF0FF30F8BD4FF034
S31508001470FF30F8BD4FF0FF30F8BD00BF2DE9F04151
S3150800148006460C460768B1F5001F3CD211F01F0F3F
S315080014903CD13161856865B93B78022B01D97B6AF5
S315080014A033B93B89B3EB541F33D97B6AB3611CE06C
S315080014B01D46B7F80A804FEA4828444510D33046F7
S315080014C02946FFF76FFF0546B0F1FF3F24D00128F4
S315080014D025D97B69984225D2C8EB0404A045EED9E4
S315080014E038462946FFF732FDB0617561B369E3B145
S315080014F003EB5423B361C4F3080330331F44F76185
S315080015000020BDE8F0810220BDE8F0810220BDE898
S31508001510F0810220BDE8F0810120BDE8F0810220BB
S31508001520BDE8F0810220BDE8F0810220BDE8F08127
S315080015302DE9F84307460668894631B9F5688DB13D
S3150800154073699D4228BF01250DE0FFF72BFF01288F
S315080015504FD9B0F1FF3F55D07369984228BF4D4621
S3150800156001D24FE001252C464FF002080134736979
S315080015709C4202D3012D3FD9444638462146FFF7FF
S3150800158011FF38B1012818BFB0F1FF3F37D0AC4280
S31508001590ECD136E02546304621464FF0FF32FFF7BC
S315080015A0E7FD0346D0F1010038BF0020B9F1000F6E
S315080015B008BF002028B1304649462246FFF7D8FD25
S315080015C003467BB9F56033697269023A93423CBFB8
S315080015D003F1FF333361337943F001033371204656
S315080015E0BDE8F883012B14BF01204FF0FF30BDE89A
S315080015F0F8830120BDE8F8830020BDE8F883BDE83C
S31508001600F8830020BDE8F8832DE9F04107460E4629
S31508001610046801292DD9636999422DD232B1204631
S3150800162011464FF0FF32FFF7A3FD40BB4FF000080D
S3150800163038463146FFF7B6FE054610B3012823D0D3
S31508001640B0F1FF3F23D0204631464246FFF790FDD2
S3150800165000BB2369B3F1FF3F1FBF01332361237921
S3150800166043F0010318BF237163699D4214D22E46C5
S31508001670DEE70220BDE8F0810220BDE8F081BDE882
S31508001680F0810020BDE8F0810220BDE8F08101204C
S31508001690BDE8F081BDE8F0810020BDE8F08100BF1B
S315080016A02DE9F04704460E46056802698369002B52
S315080016B06ED002F12007B7F5001F6CD2C7F30808F1
S315080016C0B8F1000F5CD101338361416941B92B89B7
S315080016D0B3EB571F54D8002383610420BDE8F08775
S315080016E06B89013B13EA57234AD1FFF75BFE814614
S315080016F0012853D9B0F1FF3F53D06B69984238D3CC
S3150800170026B90023A3610420BDE8F0872046616955
S31508001710FFF70EFF8146002846D0012847D0B0F1D2
S31508001720FF3F47D02846FFF773FC002845D105F14F
S31508001730300100231A46CA540133B3F5007FFAD1A3
S3150800174028464946FFF702FCE86200264FF0010AE0
S3150800175009E085F803A02846FFF75AFC80BB013646
S31508001760EB6A0133EB626B899E42F2D3EB6A9B1BF1
S31508001770EB62C4F8149028464946FFF7E7FBA061D8
S31508001780276108F130084544E5610020BDE8F08787
S315080017900420BDE8F0870420BDE8F0870220BDE8F4
S315080017A0F0870120BDE8F0870720BDE8F087022012
S315080017B0BDE8F0870120BDE8F0870120BDE8F08785
S315080017C00120BDE8F08700BF2DE9F8430446056807
S315080017D00669416AB1F1FF3F03D0FFF74FFE0346A2
S315080017E0D8B94FF0E50801274FF000092846A16946
S315080017F0FFF744FC034668B9E26982F80080EF7097
S315080018002269964209D920464946FFF749FF034609
S315080018100028EBD0042B08BF02231846BDE8F8833E
S315080018202DE9F04F89B00446D0F800B00021FFF743
S3150800183025FE002840F0AE804FF0FF3363624FF07C
S31508001840FF0AD0461F46D14644F67822C0F6000263
S31508001850029202F10C0303935846A169FFF70EFCA6
S31508001860002840F09880E5692E78002E00F09480D4
S31508001870EB7A03F03F02A271E52E04D013F0080FAD
S3150800188004D00F2A04D06762C8467BE00F2A5DD1D0
S31508001890A26A0192002A75D016F0400F06D095F874
S315080018A00DA006F0BF062369636203E0B04518BFC2
S315080018B0C84667D16B7B0493534518BFC84661D1A8
S315080018C0EA7EAB7E53EA02237ED12B7803F03F03F0
S315080018D0013B03EB430203EB8208029A02F1FF3A4B
S315080018E00121CDF814B00796464606941AF8013F2A
S315080018F0EA185478EB5C43EA042489B1FE2E58D8DA
S31508001900204601F0EBFA834606F10108019B33F8FD
S31508001910160001F0E3FA83454FD12146464603E017
S315080019204FF6FF7294424CD1039B9A45DED1DDF8FF
S3150800193014B0B046079E069C2B7813F0400F32D0A1
S3150800194089B3019A32F818306BB33DE0B8F1000F4D
S3150800195004D12846FFF706FB50451FD0216ACB7AEB
S3150800196013F0010F34D00AE013F8010F11F8012F14
S31508001970821AAB4202D0002AF6D000E082B1676232
S31508001980C846FFE720460021FFF78AFE00283FF4F5
S3150800199063AF07E022E021E004201FE000201DE0FD
S315080019A000201BE01AE0013E5FFA86F8DDF810A079
S315080019B0E8E7DDF814B0069C06E0DDF814B0069CEE
S315080019C002E0DDF814B0069CDDF810A0C846D9E799
S315080019D02A780B78D21A2B460A35CCE709B0BDE827
S315080019E0F08F00BF2DE9F04F89B0074602680192D3
S315080019F0046A836A0093E37A13F0A00F18BF0620DF
S31508001A0040F06C81009A13884BB113464FF00008DA
S31508001A1008F1010833F8022F002AF9D101E04FF046
S31508001A20000805A821460C22FFF786FA9DF81F3004
S31508001A3013F0010F00F081800023E372BB62204699
S31508001A4005A90B22FFF778FA012633464FF0070B54
S31508001A504FF07E0A4FF00009202523E0204605A90D
S31508001A600B22FFF769FA052E98BF33461AD9009B51
S31508001A70A3F1020E33464FF0100C0EE0614602F059
S31508001A80010000EB4303520813F4803F1CBF83F4A4
S31508001A90883383F021030139F1D13EF8022F002A59
S31508001AA0ECD1FFE75A4603F00F0000F1300139295F
S31508001AB088BF00F13701013A03A8104441701B0999
S31508001AC0F1D1964608AB134403F814AC62B12378F7
S31508001AD0202B0BD021464B460133734507D011F80E
S31508001AE0010F2028F8D102E04B4600E04B46072AB2
S31508001AF09FBF08A9891811F8141C013288BF294606
S31508001B00E1540133072BF2D93846FFF789FE03461D
S31508001B1020B90136642EA1D10720DFE0642E08BF64
S31508001B20072000F0DB80042B18BF184640F0D6804B
S31508001B309DF81F30E372009ABA629DF81F3013F0C1
S31508001B40020F1FBF08F10C084EF64F43C4F6C463D4
S31508001B50A3FB08231ABF4FEA930808F101084FF0C0
S31508001B6001083E6838460021FFF788FC0346D0B9CD
S31508001B700024A14601253046B969FFF77FFA0346D6
S31508001B8088B9FB691B78E52B18BF002B03D10134F4
S31508001B90A04501D10FE04C4638462946FFF780FD9F
S31508001BA003460028E7D0042B08BF072300F08E80E1
S31508001BB0002B40F08B80B8F1010800F08980396964
S31508001BC03846A1EB4811FFF759FC034600287DD19A
S31508001BD0386AFFF7C7F9009000264FF6FF7444F6F7
S31508001BE07825C0F600054FF0FF0B0198B969FFF795
S31508001BF045FA0346002869D1D7F828E0F9695FFA5B
S31508001C0088F9009B4B734FF00F02CA720E738E76DB
S31508001C10CE7609F1FF3303EB430003EB8000012284
S31508001C20334602E0604623460132A34240D000F123
S31508001C30010C3EF81030A81810F8010C01EB000A48
S31508001C400B54180A8AF80100002B3CD060460C2A6F
S31508001C50EAD9A34202D03EF810300BB949F0400940
S31508001C6081F800904FF00103019AD3703846314647
S31508001C70FFF716FD034648BBB8F10108B5D127E0C2
S31508001C80FB6903F12001002203F8012B8B42FBD1EB
S31508001C90F869396A0B22FFF74FF9FB693A6AD27A73
S31508001CA002F018021A730123019AD370002015E076
S31508001CB005EB020C1CF801CC01EB0C0A01F80CB080
S31508001CC08AF801B0C3E70C2AACD9C7E7184605E07D
S31508001CD00198B969FFF7D2F90028D1D009B0BDE853
S31508001CE0F08F00BF10B504460023C3704FF0FF33D2
S31508001CF0C362FFF7C3F938BB94F82F2294F82E3243
S31508001D0043EA022212B24AF65523CFF6FF739A42E5
S31508001D101CD104F16600FFF703F920F07F4044F276
S31508001D204613C0F25403984212D004F18200FFF71A
S31508001D30F7F820F07F4044F24613C0F25403984265
S31508001D4014BF0220002010BD042010BD032010BDC2
S31508001D50002010BD2DE9F04385B00D461746002337
S31508001D600B60FFF70FF9061EB8BF0B20C0F274818F
S31508001D7040F23C43C2F2000353F826400C20002CE4
S31508001D8000F06A812C6007F0FE07237883B160783B
S31508001D90FEF7F6FD10F0010F0AD1002F00F037818B
S31508001DA000F00400C0B2002814BF0A20002053E146
S31508001DB000232370F0B26070FEF74AFC10F0010FA2
S31508001DC018BF032040F048812FB110F0040F18BF48
S31508001DD00A2040F0418120460021FFF783FF0228B0
S31508001DE018BF002625D104F5FB7503AFADF104062F
S31508001DF04FF0000815F8043C40461BB12846FFF78B
S31508001E008FF8FFE746F8040F1035BE42F2D1ADF160
S31508001E1004054FF0030855F8046F404636B12046CE
S31508001E203146FFF75FFF012800D808E1AF42F2D13B
S31508001E30FFE7042808BF012000F00E81012888BFAB
S31508001E400D2000F2098194F83C2094F83B3043EACF
S31508001E5002231BB2B3F5007F18BF0D2040F0FC80AB
S31508001E6094F8479094F8463053EA092904D104F1C6
S31508001E705400FFF755F88146C4F8189094F8407056
S31508001E80A7707B1EDBB2012B88BF0D2000F2E48011
S31508001E9094F83D506581002D00F0BB806B1E2B42E7
S31508001EA040F0B98094F8428094F8413043EA082813
S31508001EB0A4F8088018F00F0F40F0AF8094F844009B
S31508001EC094F8433053EA002003D104F15000FFF799
S31508001ED027F894F83F2094F83E3053EA022200F09F
S31508001EE09E8007FB09F102EB18130B449842C0F0D9
S31508001EF09880C01AB0FBF5F5002D00F0948040F6E6
S31508001F00F577BD428CBF022701274FF6F57085424B
S31508001F1000F2998002356561E661324422623344F3
S31508001F20A362032F10D194F85B2094F85A3053EA31
S31508001F3002237AD1B8F1000F79D104F15C00FEF7DB
S31508001F40EFFF6062AD000EE0B8F1000F71D00A44F1
S31508001F506262022F0FBF6D0003236B4305F0010574
S31508001F6018BF05EB530505F2FF15B9EB552F62D3DC
S31508001F704FF0FF332361E36080232371032F3AD1A7
S31508001F8094F8612094F8603043EA02231BB2012BCF
S31508001F9031D12046711CFFF771F860BB002323710D
S31508001FA094F82F2294F82E3243EA022212B24AF605
S31508001FB05523CFF6FF739A421DD104F13000FEF780
S31508001FC0AFFF45F25223C4F26113984213D104F5C8
S31508001FD00570FEF7A5FF47F27223C6F24113984231
S31508001FE009D104F50670FEF79BFF206104F507701A
S31508001FF0FEF796FFE060277040F23843C2F200030E
S315080020001A88013292B21A80E280002024E0002069
S3150800201022E00D2020E00D201EE00D201CE00D2002
S315080020201AE00D2018E00D2016E00D2014E00D2012
S3150800203012E00D2010E00D200EE001200CE004282F
S315080020407FF401AFF9E702356561E6613244226241
S315080020503344A362032766E705B0BDE8F08300BFF3
S315080020602DE9F04F85B004468A4607684FF0FF0B06
S315080020705E460425D94644F67820C0F6000001904D
S3150800208000F10C0302934FF000087CE03846FEF797
S31508002090F5FF054600287BD1E2691378002B00F08E
S315080020A08480D17A01F03F01A1712E2B18BFE52B50
S315080020B061D021F02000082814BF002001205045D7
S315080020C018BF4E4659D10F294BD113F0400F06D0F1
S315080020D092F80DB003F0BF032169616203E09E42E6
S315080020E018BF4E4649D1557B5D4518BF4E4644D16B
S315080020F0D4F828C0D07E917E51EA002152D11178B9
S3150800210001F03F01013901EB410601EB8606019812
S31508002110411E4FF0010E0393A3467446DDF808E00E
S3150800212011F8013FD0184078D35C43EA002334B154
S31508002130FE2E34D82CF816301C46013603E04FF62E
S31508002140FF7083422DD17145EAD1039B5C46127814
S3150800215012F0400F1FD0FE2E98BF2CF816801AD901
S3150800216020E010461EB9FEF7FDFE58451FD04FF079
S31508002170FF3363621BE04E46FFE720464146FFF702
S315080021808FFA054620B9A16900297FF47FAF75B19A
S315080021900023A3610BE0013BDEB2AB46EDE75C46EC
S315080021A000E05C46AB464E46E7E70425F0E72846DE
S315080021B005B0BDE8F08F00BFCA7E8B7E43EA0223D6
S315080021C00278032A01BF487D0A7D42EA002243EAD3
S315080021D002431846704700BF2DE9F04F87B0824684
S315080021E00D46006800900B782F2B18BF5C2B05D185
S315080021F015F8013F2F2B18BF5C2BF9D00023CAF81E
S3150800220008302B781F2B09D8DAF820308022DA72AA
S3150800221050460021FFF732F9034682E14FF00108E4
S3150800222044F6E419C0F6000944F6F011C0F60001B8
S31508002230049144F6F812C0F600020592DAF828B0BE
S3150800224028782F2818BF1F2809D95C280AD0ABF18F
S3150800225002072E4644461CE05C2B15D104E00024F8
S31508002260424601E00024424615442B782F2B18BF1E
S315080022705C2B2CD12B465A1C15465B782F2B18BF86
S315080022805C2B24D11346F6E7B2F5807F00F0448133
S315080022901446414600F0FCFD0146002800F03C814A
S315080022A07F2809D8222900F037814A4612F8013FCB
S315080022B013B19842FAD12FE127F8021F621C16F8CB
S315080022C0013F18462F2B18BF1F2BC5D8CCE71F2850
S315080022D094BF04260026002C00F00B8104F100436D
S315080022E0013B5A003BF813302E2B18BF202B40F029
S315080022F0F480931C5B4407E033F8042C023B2E2A37
S3150800230018BF202A40F0E980013CF5D1F1E04FF0F2
S31508002310200003F8010B8B42F9D1BBF80030202BC3
S3150800232018BF2E2B40F0E98058460023013330F8B9
S31508002330021F202918BF2E29F8D0002B00F0DE80B6
S3150800234046F00306DAE0013C05D108210391002294
S315080023500192029205E0023A32F8021C2E29F2D1C5
S31508002360F3E75F1C3BF81300002861D0202808D04B
S31508002370E31B18BF01232E2814BF002203F0010215
S315080023801AB146F003063B46EBE70199039ABC42AD
S3150800239018BF914214D30B2A03D146F00306029ABA
S315080023A049E00BB146F00306A74243D802988300DA
S315080023B0DBB2029323460B21039108220192D0E750
S315080023C07F280DD9002100F063FD0346002800F0A0
S315080023D0A5800598034413F8800C46F0020650B110
S315080023E001462B2807D0049A12F8013F002B00F06B
S315080023F08C809942F8D146F003065F2010E00299D6
S3150800240041F0020102910BE0A0F161039BB2192B86
S315080024109FBF029A42F001020292203898BF80B20A
S31508002420DAF82030019958543B460131019198E772
S31508002430029A00E0029ADAF820301978E52904BFF2
S3150800244005211970039B082B02BF9200D2B2029293
S31508002450029800F00C030C2B03D000F00302032AA9
S3150800246001D146F0020616F0020F0AD1029901F0D0
S315080024700302012A08BF46F01006042B08BF46F0DF
S315080024800806DAF82030DE725046FFF7C9F9DAF89E
S315080024902030DA7A034648B1042842D102F0040310
S315080024A0DBB2002B14BF034605233AE012F0040FF3
S315080024B037D19AF8063013F0100F0CD0DAF810302E
S315080024C0C3F3080303F1300100980144FFF774FED3
S315080024D0CAF80800B2E6052323E067000BEB0702FB
S315080024E04FF000032BF81430DAF8203003F10B0113
S315080024F00DE700232BF814300EE000235F4437F86D
S31508002500021C2E293FF421AF1DE7A0F141039BB21F
S31508002510192B7FF674AF77E7062302E046F002062A
S3150800252069E7184607B0BDE8F08F00BF10B584B05C
S3150800253001900091144604A840F8041DFEF722FDF8
S315080025400028B8BF0B202CDB40F23C43C2F2000344
S3150800255053F820300BB100221A70019BCBB1002230
S315080025601A70019A40F23C43C2F2000343F8202055
S31508002570D2F1010238BF0022012C0CBF144642F0EA
S31508002580010400206CB9684601A90022FFF7E2FBA6
S3150800259007E040F23C43C2F20003002243F8202041
S315080025A0104604B010BD00BF2DE9F04393B0019169
S315080025B015460446002800F0A1800023036002F0B7
S315080025C01F0601A806A93246FFF7C4FB002840F0FB
S315080025D09780069B079303AB0F9340F23823C2F20A
S315080025E00003119307A80199FFF7F6FD0346002893
S315080025F040F08C800F9B93F90B30002B80F2818082
S3150800260083E053B1042B40F08D8007A8FFF7EAF961
S3150800261046F00806034640B184E09DF8223013F0E0
S31508002620110F78D115F0040F77D116F0080F48D09E
S315080026300E9B00259D73DD736121197448225A7417
S315080026400E9B9D75DD7519765A7620220E9BDA72D9
S31508002650DDF818800E9F40463946FFF7ADFD8146E6
S31508002660404639462A46FEF717FE0E9B1D775D77CC
S315080026709D77DD770122069BDA70B9F1000F20D02D
S31508002680069BDD6A07A849460022FEF7BDFF0346FA
S31508002690002847D106982946FEF7F0FC034609F1BB
S315080026A0FF31069AD1600BE09DF8223013F0100F27
S315080026B035D115F0020F04D013F0010F31D100E027
S315080026C083BB16F0080F18BF46F02006069DEB6A76
S315080026D023620E9F676228463946FFF76DFDA060A4
S315080026E007F11C00FEF71CFCE060002060746061C6
S315080026F0E06126742560EB88A38014E0092012E0C7
S3150800270011E015F01C0F88D1CEE7062315F01C0F33
S315080027107FF477AFD4E7072304E0082302E0042315
S3150800272000E00723184613B0BDE8F0832DE9F04F03
S3150800273085B004460F4690461E460023336003A91B
S31508002740FEF74CFC002840F0A880607C002840F08A
S31508002750A880237C13F0010F08BF072000F0A18092
S31508002760E5686369ED1AA84538BF4546002D00F0AF
S31508002770958004F1280301936369C3F30802002ACC
S3150800278071D1039AB2F80AA00AF1FF3A1AEA532A53
S3150800279012D10BB9A06803E02046A169FEF702FE34
S315080027A0012802D8022060747BE0B0F1FF3F02D115
S315080027B00120607475E0A061DDF80C804046A169CF
S315080027C0FEF7C4FB814610B90220607469E0D14463
S315080027D05FEA552B25D0B8F80A300BEB0A029A4265
S315080027E088BFCAEB030B98F8010039464A465B4690
S315080027F0FEF7D0F810B10120607452E0237C13F084
S31508002800400F0BD0E369C9EB0300834506D907EBF4
S31508002810402001994FF40072FEF78EFB4FEA4B2BCE
S315080028202FE0E2694A451CD0237C13F0400F0DD0F7
S3150800283098F8010001990123FEF7FAF810B1012072
S3150800284060742EE0237C23F040032374039B58789E
S3150800285001994A460123FEF79DF810B101206074DC
S315080028601FE0C4F81C906169C1F30801C1F5007B3B
S315080028705D4538BFAB462831384621445A46FEF7EF
S315080028805BFB5F4463695B44636133685B44336045
S31508002890B5EB0B057FF470AF02E002E0002000E024
S315080028A0002005B0BDE8F08F2DE9F04F85B004464D
S315080028B00F4615461E460023336003A9FEF78EFB16
S315080028C0002840F0C580607C002840F0C280237C48
S315080028D013F0020F08BF072000F0BB806369DD42D2
S315080028E028BFDD43002D00F0AD8004F128030193D5
S315080028F06369C3F30802002A40F08280039AB2F89B
S315080029000AB00BF1FF3B1BEA532B1DD133B9A06864
S3150800291058B920460021FEF70BFE03E02046A169C0
S31508002920FEF706FE002800F08D80012802D102205D
S3150800293060748EE0B0F1FF3F02D10120607488E038
S31508002940A061A36803B9A060237C13F0400F0ED0E2
S31508002950039B58780199E2690123FEF769F810B1DB
S315080029600120607475E0237C23F040032374DDF8AE
S315080029700C804046A169FEF7E9FA814610B90220A3
S31508002980607466E0D9445FEA552A25D0B8F80A305B
S315080029900AEB0B029A4288BFCBEB030A98F80100B0
S315080029A039464A465346FEF743F810B1012060748B
S315080029B04FE0E369C9EB03018A450AD9019807EB99
S315080029C041214FF40072FEF7B7FA237C23F0400347
S315080029D023744FEA4A2A25E0E3694B450ED062691B
S315080029E0E3689A420AD298F8010001994A460123F7
S315080029F0FDF7D0FF10B1012060742AE0C4F81C90DE
S31508002A006069C0F30800C0F5007A554538BFAA4684
S31508002A102830204439465246FEF78EFA237C43F086
S31508002A20400323745744636953446361E2689A42D6
S31508002A302CBFE260E360336853443360B5EB0A05A4
S31508002A407FF456AF237C43F020032374002000E074
S31508002A50FFE705B0BDE8F08F70B582B004460E46B4
S31508002A600A2902D10D21FFF7F7FF6368002B14DB53
S31508002A705D1C23441E733C2D0BDD214651F80C0BBF
S31508002A802A4601ABFFF710FF019BED1A18BF6FF03E
S31508002A9000056560A3680133A36002B070BD00BF7E
S31508002AA030B583B0044601A9FEF798FA002840D14C
S31508002AB0237C13F0200F08BF00203DD013F0400FF1
S31508002AC00CD0019B587804F12801E2690123FDF72F
S31508002AD0AFFF78BB237C23F0400323740198216A57
S31508002AE0FEF7CCFA40BB656AEB7A43F02003EB723B
S31508002AF020682946A268FEF7CFFBE3682B771A0AF7
S31508002B006A771A0CAA771B0EEB770023AB75EB7561
S31508002B1061222A7648226A76AB74EB740122019BFD
S31508002B20DA700198FEF7C8FA237C23F02003237491
S31508002B3002E001E00120FFE703B030BD10B582B026
S31508002B400446FFF7ADFF034638B9204601A9FEF74C
S31508002B5045FA034608B900222260184602B010BD9D
S31508002B6070B582B004460D4601A9FEF737FA00286B
S31508002B7040F0AB80607C002840F0A880E368AB4258
S31508002B8006D2227C02F00202D2B2002A08BF1D46F3
S31508002B906269002363610020002D00F09780019B85
S31508002BA05E8976026AB1013A691EB1FBF6F1B2FB9B
S31508002BB0F6F3994205D373421A406261AD1AA169C8
S31508002BC012E0A16879B92046FEF7B2FC0146012851
S31508002BD004BF0220607479D0B1F1FF3F04BF012021
S31508002BE0607473D0A160A161002937D0B54225D998
S31508002BF0227C12F0020F05D02046FEF799FC01460A
S31508002C0020B91AE02046FEF7CDFB0146B1F1FF3F99
S31508002C1002D10120607459E0012903D9019A526949
S31508002C20914202D30220607450E0A1616269324485
S31508002C306261AD1BAE42DBD300E0354662692A44C9
S31508002C406261C5F308025AB10198FEF77FF910B917
S31508002C50022060743AE000EB552502E0002500E00A
S31508002C6000256369C3F3080313B3E269AA421FD0B8
S31508002C70237C13F0400F0ED0019B587804F12801ED
S31508002C800123FDF7D5FE10B1012060741EE0237CF8
S31508002C9023F040032374019B587804F128012A463F
S31508002CA00123FDF777FE10B1012060740EE0E5619F
S31508002CB06369E268934298BF002007D9E360237CE2
S31508002CC043F020032374002000E0FFE702B070BD44
S31508002CD030B591B010AB43F83C0D0D46184605A922
S31508002CE00022FFF737F80446C8B902AB0D9340F245
S31508002CF03823C2F200030F9305A80199FFF76CFA6F
S31508002D00044660B90D9B93F90B30002BB8BF062417
S31508002D1005DB25B105A82946FEF7CAFAFFE72046CE
S31508002D2011B030BD70B59CB01CAB43F86C0D18469D
S31508002D3005A90222FFF70EF8059B11930346002802
S31508002D4051D102AB199340F23823C2F200031B9308
S31508002D5011A80199FFF740FA0346002843D1199BA9
S31508002D6093F90B30002BB8BF06233CDB9DF84A408D
S31508002D7014F0010F18BF072335D11CE006960895F5
S31508002D8006A80021FEF77AFB034660BB06A80021C9
S31508002D90FFF766F9034628B3042815D023E011A8DF
S31508002DA029460022FEF730FC0346E3B90598FEF7EC
S31508002DB083F9034617E0059E30461899FFF7FCF994
S31508002DC0054614F0100FD9D111A8FEF7FDFC0346ED
S31508002DD0D0F1010038BF0020002D08BF00200028D0
S31508002DE0E3D0DCE7072318461CB070BD2DE9F04395
S31508002DF083B081469046054600244E1E012711E001
S31508002E00404601A93A466B46FFF790FC009B012B0A
S31508002E100AD19DF804300D2B04D005F8013B013486
S31508002E200A2B01D0A642EBDC00232B709C4214BF70
S31508002E304846184603B0BDE8F08300BF10B594B005
S31508002E400191002302930393017839B1044601A83E
S31508002E50FFF702FE14F8011F0029F8D1029A002A8A
S31508002E600BDB019804A96B46FFF71EFD40B9009BD2
S31508002E70029A9A4207D1039807E04FF0FF3004E020
S31508002E804FF0FF3001E04FF0FF3014B010BD00BF27
S31508002E907F2821D941B9C7281EBF44F64432C0F657
S31508002EA0000201230AD112E0FF2814D8803844F61C
S31508002EB04433C0F6000333F81000704732F8021F97
S31508002EC0814205D001339BB2802BF7D100E0002365
S31508002ED08033D8B270470020704700BFF0B444F67C
S31508002EE08822C0F6000244F64443C0F60003B0F553
S31508002EF0805F38BF1A460432164632F8043CD3F1CE
S31508002F00010138BF0021984238BF41F0010100296C
S31508002F1035D132F8021C0C0AC9B25D18A84228DA63
S31508002F20082C2CD8DFE804F005090F1215181B1E0B
S31508002F302100C71A36F8170021E0C31A03F0010367
S31508002F40C01A80B21BE0103880B218E0203880B270
S31508002F5015E0303880B212E01A3880B20FE0083037
S31508002F6080B20CE0503880B209E0A0F5E35080B298
S31508002F7005E00432002CBFD106EB4102BBE7F0BCEA
S31508002F80704700BF08B500F039FF00F0BDFA01F040
S31508002F90BBF901F09BF900F03BFB00F00FF800F0DD
S31508002FA0A1FA08BD08B500F0B1FA01F0C9F900F0B8
S31508002FB071FC00F013F800F06FFA08BD10B500F0C8
S31508002FC087F800F049FF40F20104C2F20004012329
S31508002FD0237001F0B5F80023237010BD08B540F240
S31508002FE04040C2F2000001F03FF801280BD140F240
S31508002FF00103C2F2000301221A7040F24040C2F2F5
S31508003000000000F085F840F24040C2F2000001F0EE
S31508003010E1F801280BD140F20103C2F200030022B5
S315080030201A7040F24040C2F2000000F071F808BD84
S31508003030704700BF38B505460C4640F20103C2F298
S3150800304000031B78012B02D1C9B200F0B9FF40F288
S315080030500103C2F200031B781BB92846E1B201F04E
S3150800306085F800F04DF838BD40F20103C2F20003BE
S315080030701878022806D0032806D001280CBF082095
S3150800308040207047002070470020704740F2010337
S31508003090C2F200031878022806D0032806D00128B1
S315080030A00CBF08204020704700207047002070475A
S315080030B008B500F01BF808BD40F28043C2F20003D1
S315080030C0FE22DA7018710222A3F84420704700BF66
S315080030D040F28043C2F2000300221A709A6483F811
S315080030E04320A3F844209A705A70704740F28043F0
S315080030F0C2F200031878003018BF0120704700BFDD
S3150800310040F28043C2F20003002283F8432070474E
S3150800311038B504460178FF2925D100F093FA18B985
S315080031201020FFF7C9FF98E140F28044C2F200047C
S315080031300023637001252570FF22E2701022227198
S315080031406371FFF791FFA071FFF7A0FFE071FFF72A
S315080031509DFF000A20726572A5720823A4F8443000
S3150800316001F0B4F879E140F28043C2F200031B781B
S31508003170012B40F09081C939352900F26B81DFE8CF
S3150800318011F0DB00690169016501690169015901ED
S31508003190FC0042012F0169016901690169016901A0
S315080031A069016901690169016901690169016901C1
S315080031B069016901690169016901690169016901B1
S315080031C069016901690169016901690169016901A1
S315080031D06901690169017F005400360073006901BD
S315080031E069016901A1006901B900BD00CE004578F1
S315080031F0FFF73AFF0138854203DD2220FFF75CFF1F
S315080032002BE140F28045C2F20005281DA96C6278C0
S3150800321000F012FEFF23EB706278AB6C1344AB64CC
S3150800322063780133A5F8443017E14578FFF71CFFAA
S315080032300138854203DD2220FFF73EFF0DE1616874
S3150800324040F28045C2F20005A964281D627800F0A4
S31508003250F3FDFF23EB706278AB6C1344AB646378C1
S315080032600133A5F84430F8E040F28043C2F2000387
S31508003270FF22DA7042689A640122A3F84420ECE03F
S3150800328040F28043C2F20003FF22DA709B6C40686A
S3150800329040B11844002213F8011B0A44D2B28342F3
S315080032A0F9D100E0002240F28043C2F20003C3F8DD
S315080032B0072001221A7100225A719A710822A3F86E
S315080032C04420CAE040F28043C2F20003FF22DA70CB
S315080032D044F63862C0F600029A6400221A715A71DE
S315080032E09A710721D9711A725A729A720822A3F82A
S315080032F04420B2E00020FFF7DFFEAEE040F2804354
S31508003300C2F20003FF22DA7000221A715978597145
S315080033109A71DA711A720622A3F844209DE040F2E7
S315080033208043C2F2000300221A705A70FF22DA7034
S315080033300122A3F8442090E040F28043C2F2000341
S315080033409D6CFFF791FE411E2846621C00F0C2FFE5
S3150800335018B93120FFF7B0FE7FE040F28044C2F290
S315080033600004FF23E370A56CFFF77EFE013D2844A9
S31508003370A0640123A4F844306FE04578FFF774FE93
S315080033800238854203DD2220FFF796FE65E040F20B
S315080033908043C2F20003FF22DA700122A3F8442018
S315080033A0617839B900F0A6FF002856D13120FFF719
S315080033B083FE52E040F28043C2F20003986CA21CDE
S315080033C000F088FF18B93120FFF776FE45E040F295
S315080033D08043C2F2000361789A6C0A449A643CE01E
S315080033E040F28044C2F20004FF23E37000252571F1
S315080033F06571FFF739FEA071E571257265720723BD
S31508003400A4F8443029E040F28043C2F20003986CE5
S31508003410616800F063FF18B93120FFF74DFE1CE024
S3150800342040F28043C2F20003FF22DA700122A3F8B9
S31508003430442012E000F0E6FC40F28043C2F20003AA
S31508003440FF22DA700122A3F8442006E03120FFF7B4
S3150800345033FE02E02020FFF72FFE40F28043C2F23F
S31508003460000393F84330012B02D11020FFF724FE06
S3150800347040F28043C2F20003B3F844100BB2002BAB
S3150800348009DD40F28040C2F20000012380F8433093
S315080034900330FFF7CFFD38BD08B5FFF709FE012851
S315080034A01FD000F0CFF8E0B140F2CC43C2F20003DF
S315080034B01B78012B15D100F055FF40F2D043C2F21C
S315080034C000031B6803F5FA7398420AD340F2CC430B
S315080034D0C2F2000300221A7000F0BEF808B900F024
S315080034E091FC08BD08B540F2CC43C2F200030122A4
S315080034F01A7000F037FF40F2D043C2F2000318609A
S31508003500FFF7CAFF08BD00BF704700BF704700BF7E
S3150800351000F00F03092802D903F13700704703F1B9
S31508003520300040F20403C2F200031B6803445B78D0
S3150800353003F00303022B08BF2038C0B2704700BF50
S3150800354038B505460C460009FFF7E2FF207005F07E
S315080035500F00FFF7DDFF60700023A370204638BD1B
S3150800356030B4024603464CF6CD40CCF6CC40013189
S31508003570A0FB0343DB08FAD1002301F801394CF616
S31508003580CD45CCF6CC450846A5FB0243DB0803EB44
S315080035908304A2EB4402303201F801291A46002BB3
S315080035A0F1D130BC704700BFF0B440F20403C2F258
S315080035B000031F6800231C46C15C7A18527802F083
S315080035C00302022A08BF2039C9B2A1F13002D2B2D9
S315080035D0A1F13A05EDB2162A94BF00260126062D5A
S315080035E08CBF354646F0010565B9092A84BFA1F1A5
S315080035F03702D2B22401E4B22244D4B20133022BF8
S31508003600DAD101E0002000E02046F0BC704700BF98
S3150800361008B540F21453C2F2000300221A7040F2B1
S315080036202050C2F2000044F64061C0F60001FEF7E1
S315080036307DFF30B144F64460C0F60000772100F003
S31508003640D9FB08BD40F21453C2F200031878D0F132
S31508003650010038BF0020704708B5FFF729FD01288B
S315080036600FD040F21453C2F200031B785BB9FCF783
S315080036706FFD012809D140F21453C2F200031870F5
S3150800368008BD002008BD002008BD002008BD00BFF9
S31508003690027840F20403C2F200031B6899184978BD
S315080036A001F00301022908BF203A532A0ED14078B7
S315080036B003445B7813F0040F0AD031280AD0322865
S315080036C00AD0332814BF032002207047032070470E
S315080036D003207047002070470120704770B50446E4
S315080036E00230FFF761FF0646054604342046FFF719
S315080036F05BFF3044C6B2013DADB20234012DF5D8A8
S315080037002046FFF751FFF643F6B2864214BF002063
S31508003710012070BD2DE9F04115460F4604460029E3
S3150800372018BF002807D144F64460C0F6000040F2EE
S31508003730612100F05FFB2046FFF7AAFF0646032833
S3150800374008BF002000F0A2802046FFF7C7FF002828
S3150800375000F08C80012E29D016B1022E53D088E0B5
S31508003760A01CFFF721FF8046201DFFF71DFF06025C
S315080037703E60A01DFFF718FF3044386004F10806C4
S31508003780A8F103081FFA88F84046002D7ED00FFAE4
S3150800379088F7002F6FDD00243046FFF705FF285510
S315080037A002360134A4B2BC42F6DB66E0A01CFFF781
S315080037B0FBFE8046201DFFF7F7FE06043E60A01DAF
S315080037C0FFF7F2FE06EB00263E6004F10800FFF75D
S315080037D0EBFE3044386004F10A06A8F104081FFA23
S315080037E088F84046002D51D00FFA88F7002F46DD9D
S315080037F000243046FFF7D8FE285502360134A4B215
S31508003800BC42F6DB3DE0A01CFFF7CEFE8046201D3D
S31508003810FFF7CAFE06063E60A01DFFF7C5FE06EBCB
S3150800382000463E6004F10800FFF7BEFE06EB0026E0
S315080038303E6004F10A00FFF7B7FE3044386004F131
S315080038400C06A8F105081FFA88F84046F5B10FFAE4
S3150800385088F7002F17DD00243046FFF7A5FE285508
S3150800386002360134A4B2BC42F6DB0EE04FF6FF7016
S315080038700CE000200AE0404608E0404606E04046E4
S3150800388004E0404602E0404600E0404600B2BDE89B
S31508003890F08100BFF8B540F21453C2F200031B785A
S315080038A0002B00F0A382012B41D100F00FFDFCF79D
S315080038B075FC44F65C60C0F60000FCF7C1FC44F6F3
S315080038C08060C0F60000FCF7BBFCFCF761FC014613
S315080038D0CF480122FEF768FE48B144F6A860C0F654
S315080038E00000FCF7ADFC0120FCF79AFCF8BD44F695
S315080038F0B060C0F60000FCF7A3FC44F6B860C0F65A
S315080039000000FCF79DFC44F6DC60C0F60000FCF7FE
S3150800391097FC40F21853C2F2000300221A605A605C
S3150800392040F21453C2F2000302221A70F8BD022BA9
S3150800393040F0708140F22054C2F2000440F678103C
S31508003940C2F200004FF4807104F50C72FFF74EFACC
S3150800395094F841329BB144F6A860C0F60000FCF723
S315080039606FFC0220FCF75CFC04F50C70FFF7E6F828
S3150800397040F21453C2F2000300221A70F8BD002860
S3150800398000F0B98040F67811C2F20001084601F548
S31508003990C0710022FFF7BEFE0446B0F1FF3F12D108
S315080039A044F6A860C0F60000FCF74AFC0320FCF7C2
S315080039B037FC9748FFF7C2F840F21453C2F20003E7
S315080039C000221A70F8BD002840F3958040F218537B
S315080039D0C2F200035B6863B940F21853C2F20003EF
S315080039E040F67812C2F20002D2F880211A605860B6
S315080039F081E040F67812C2F2000240F21851C2F293
S31508003A00000109681944D2F880218A4206D140F299
S31508003A101852C2F20002034453606CE044F6B060E8
S31508003A20C0F60000FCF70CFC44F60C70C0F600006B
S31508003A30FCF706FC40F21856C2F2000640F2D445DE
S31508003A40C2F2000570682946FFF78AFD2846FCF78A
S31508003A50F7FB44F61870C0F60000FCF7F1FB376870
S31508003A60380E2946FFF76CFDC7F30740A91CFFF778
S31508003A7067FDC7F30720291DFFF762FDF8B2A91DE8
S31508003A80FFF75EFD2846FCF7DBFB44F6BC70C0F684
S31508003A900000FCF7D5FB3068716800F01FFC90B990
S31508003AA044F6A860C0F60000FCF7CAFB0520FCF740
S31508003AB0B7FB5748FFF742F840F21453C2F2000327
S31508003AC000221A70F8BD44F6B060C0F60000FCF794
S31508003AD0B7FB44F6DC60C0F60000FCF7B1FB40F229
S31508003AE01853C2F2000340F67812C2F20002D2F866
S31508003AF080211A605C6040F22053C2F20003D3F8BA
S31508003B004422D3F83C329A4240F070814048002162
S31508003B10FFF726F890B144F6A860C0F60000FCF757
S31508003B208FFB0420FCF77CFB3948FFF707F840F2C7
S31508003B301453C2F2000300221A70F8BD40F218535B
S31508003B40C2F200035B68002B54D044F6B060C0F69E
S31508003B500000FCF775FB44F60C70C0F60000FCF795
S31508003B606FFB40F21855C2F2000540F2D444C2F287
S31508003B70000468682146FFF7F3FC2046FCF760FB63
S31508003B8044F61870C0F60000FCF75AFB2E68300E93
S31508003B902146FFF7D5FCC6F30740A11CFFF7D0FC6A
S31508003BA0C6F30720211DFFF7CBFCF0B2A11DFFF7D6
S31508003BB0C7FC2046FCF744FB44F6BC70C0F6000080
S31508003BC0FCF73EFB2868696800F088FB90B944F664
S31508003BD0A860C0F60000FCF733FB0520FCF720FBC5
S31508003BE00B48FEF7ABFF40F21453C2F20003002263
S31508003BF01A70F8BD44F6B060C0F60000FCF720FB6A
S31508003C0040F21453C2F2000303221A70F8BD00BF33
S31508003C1050070020032B40F0E98040F22054C2F2FE
S31508003C20000440F67810C2F200004FF4807104F5E3
S31508003C300C72FFF7DBF894F841329BB144F6347006
S31508003C40C0F60000FCF7FCFA0220FCF7E9FA04F5D6
S31508003C500C70FEF773FF40F21453C2F20003002201
S31508003C601A70F8BD00287CD040F67812C2F200021D
S31508003C70104602F5C07102F58072FFF74BFD064645
S31508003C80B0F1FF3F12D144F65870C0F60000FCF7B9
S31508003C90D7FA0320FCF7C4FA5548FEF74FFF40F25F
S31508003CA01453C2F2000300221A70F8BD002858DD2A
S31508003CB044F67C70C0F60000FCF7C2FA40F2D44421
S31508003CC0C2F2000430462146FFF74AFC2046FCF7BC
S31508003CD0B7FA44F68C70C0F60000FCF7B1FA40F665
S31508003CE07815C2F2000595F883012146FFF728FCEE
S31508003CF095F88201A11CFFF723FC95F88101211D87
S31508003D00FFF71EFC95F88001A11DFFF719FC204658
S31508003D10FCF796FA44F6BC70C0F60000FCF790FA79
S31508003D20D5F88001314605F5807200F0D3FA90B9CE
S31508003D3044F6A860C0F60000FCF782FA0620FCF7F5
S31508003D406FFA2B48FEF7FAFE40F21453C2F200034C
S31508003D5000221A70F8BD44F6B060C0F60000FCF701
S31508003D606FFA40F22053C2F20003D3F84422D3F884
S31508003D703C329A423AD144F6A470C0F60000FCF7E9
S31508003D805FFA00F0B7FA90B944F6A860C0F60000EA
S31508003D90FCF756FA0720FCF743FA1548FEF7CEFE5D
S31508003DA040F21453C2F2000300221A70F8BD44F61A
S31508003DB0B060C0F60000FCF743FA44F6C070C0F6DF
S31508003DC00000FCF73DFA0A48FEF7B8FE44F6D8703C
S31508003DD0C0F60000FCF734FA40F21453C2F20003AE
S31508003DE000221A70FCF7F2F900F00CF8F8BD00BFD3
S31508003DF05007002008B5FFF789FBFCE708B500F077
S31508003E004FFD08BD10B500F06DFAA0B1FFF710F927
S31508003E1000F08EFA00F06AFA20F0604020F07F0089
S31508003E204EF60853CEF20003186000F05FFA4468B5
S31508003E3000F038FDA04710BD70B5561EB6B24AB19F
S31508003E404C1E0E44451A14F8013F2B55FFF75EFB2E
S31508003E50B442F8D170BD00BF2DE9F047002345F202
S31508003E602C00C0F600004FF4FA7448F6A04113F887
S31508003E700080C21892F801C008EB0C0202FB04424B
S31508003E8091FBF2F902FB191636B94D4609F1FF32D4
S31508003E9092B2B2F5806F03D30233242BE7D187E0C1
S31508003EA04746E2464FF4C843C4F2000300225A616B
S31508003EB01A6842F400421A601B6813F4004F09D0CE
S31508003EC04FF4C844C4F20004FFF720FB236813F438
S31508003ED0004FF9D14FF4C843C4F200031A6822F020
S31508003EE002021A601A6842F001021A605B6813F04F
S31508003EF0010F09D14FF4C844C4F20004FFF706FBCA
S31508003F00636813F0010FF9D0013F0AF1FF36360551
S31508003F1046EA0747013D3D434FF4C843C4F2000350
S31508003F20DD611A6822F001021A605B6813F0010F5E
S31508003F3009D04FF4C844C4F20004FFF7E7FA6368EF
S31508003F4013F0010FF9D14FF4C843C4F20003D3F8B4
S31508003F50002242F00102C3F80022D3F81C2222F004
S31508003F600102C3F81C22D3F80C2242F00102C3F85E
S31508003F700C220022C3F84022C3F84422D3F80422B4
S31508003F8022F00102C3F80422D3F8142222F0010217
S31508003F90C3F81422D3F81C2242F00102C3F81C22EB
S31508003FA0D3F8002222F00102C3F80022BDE8F08708
S31508003FB045F20400C0F60000E221FFF71BFF71E797
S31508003FC038B504460D464FF4C843C4F200039B684F
S31508003FD013F0806F07D145F20400C0F6000040F2E6
S31508003FE02111FFF707FF4FF4C843C4F20003D3F8C3
S31508003FF0802102F00102C3F88021D3F8802142F023
S315080040007C4242F40012C3F88021C3F88451E17857
S31508004010A278120442EA016221780A43617842EAE8
S315080040200122C3F88821E179A279120442EA0162E1
S3150800403021790A43617942EA0122C3F88C21D3F82F
S31508004040802142F00102C3F880219B6813F0806F3B
S3150800405009D14FF4C844C4F20004FFF757FAA3681D
S3150800406013F0806FF9D038BD4FF4C843C4F200038B
S31508004070DB6813F0030F39D04FF4C843C4F20003CA
S31508004080D3F8B02140F26763B3EB525F18BF002044
S3150800409023D14FF4C843C4F20003D3F8B821027001
S315080040A0D3F8B821120A4270D3F8B821120C8270DC
S315080040B0D3F8B821120EC270D3F8BC210271D3F816
S315080040C0BC21120A4271D3F8BC21120C8271D3F8B2
S315080040D0BC311B0EC3710120FFE74FF4C843C4F27D
S315080040E00003DA6842F02002DA6070470020704761
S315080040F010B54FF48843C4F200031B8803F080030D
S315080041009BB2B3B14FF48843C4F2000398801B886E
S3150800411003F080039BB273B94FF48844C4F20004D9
S31508004120FFF7F4F9238803F080039BB2002BF7D03E
S3150800413003E0002010BD012010BD012010BD00BF06
S315080041404FF48843C4F2000300221A819A811A8226
S315080041509A821A8340F271221A819A8992B242F49B
S31508004160005242F00C029A81704700BF2DE9F041D7
S3150800417006460C46402906D945F25000C0F600000E
S315080041808D21FFF737FE2046FFF7B2FF012806D03C
S3150800419045F25000C0F600009121FFF72BFE254698
S315080041A0ACB1002445F25007C0F600074FF09A0854
S315080041B0FFF7ACF9305DFFF79BFF012803D03846BF
S315080041C04146FFF717FE0134A3B2AB42F0D3BDE870
S315080041D0F08100BF10B540F6FC23C2F200031B783D
S315080041E05BBB4FF48843C4F200031B8803F020032B
S315080041F09BB2002B56D04FF48843C4F200039A882A
S3150800420092B240F60433C2F200031A7012F0FF0F9E
S315080042104AD000F0A7F840F60033C2F2000318604F
S3150800422040F64833C2F200030020187040F6FC231B
S31508004230C2F2000301221A7010BD40F64833C2F2DA
S3150800424000031A784FF48843C4F200031B8803F06E
S3150800425020039BB263B34FF48843C4F200039C88DF
S3150800426040F60433C2F2000399184C700132D2B2F8
S3150800427040F64831C2F200010A701B78934215D104
S315080042801149FFF7D9FD40F6FC23C2F200030022CC
S315080042901A70012010BD40F6FC23C2F2000300206C
S315080042A0187010BD002010BD002010BD002010BDE4
S315080042B000F058F840F60033C2F200031B68643376
S315080042C09842E8D8002010BD050B002008B500F07C
S315080042D05BF908BD08B500F065F908BD08B500F03A
S315080042E089F908BD08B500F071FA08BD08B500F0EF
S315080042F0C7FA08BD08B500F03DFA10B100F09AFA01
S3150800430008BD002008BD00BF4EF21003CEF2000320
S3150800431000221A6041F63F11C0F2010159609A6005
S315080043200521196040F64C33C2F200031A60704743
S315080043304EF21003CEF2000300221A60704700BF47
S315080043404EF21003CEF200031B6813F4803F1FBF22
S3150800435040F64C33C2F200031A68013218BF1A60DD
S31508004360704700BF08B5FFF7EBFF40F64C33C2F2C3
S315080043700003186808BD00BF4FF40053C4F20203D7
S315080043801A6942F080021A61704700BFF8B50746FD
S315080043900024254645F27806C0F60006FFF7B6F86B
S315080043A0A359BB420ED8311949680B449F4209D21A
S315080043B045F27803C0F6000305EB450203EB8203DA
S315080043C0187AF8BD01350C349C2CE7D1FF20F8BDCE
S315080043D02DE9F84380460068FFF7D8FFFF285CD030
S315080043E04FF40053C4F2020340F22312C4F2675298
S315080043F05A6048F6AB12CCF6EF525A603422DA60AD
S31508004400DB6813F0010F04D0FFF7B6FF0020BDE804
S31508004410F8834FF40053C4F202031A6942F001020A
S315080044201A61002508F104094FF40054C4F2020485
S31508004430D8F80030EF1859F80560B2B2EA52E368C6
S3150800444013F0010F05D0FFF761F8E36813F0010FC9
S31508004450F9D1330C7B80E36813F0010F05D0FFF721
S3150800446055F8E36813F0010FF9D13B68B34204D15C
S315080044700435B5F5007FDBD101E0002400E0012416
S315080044804FF40053C4F202031A6922F001021A61BA
S31508004490FFF772FF2046BDE8F8830020BDE8F883E1
S315080044A038B504460D4640F65033C2F2000398422A
S315080044B009D04FF4C043C0F6000399420BD0FFF76A
S315080044C087FF20B917E040F65454C2F20004C5F33A
S315080044D0080393B903E040F65034C2F20004236897
S315080044E09D420CD0204640F8045B29464FF40072E2
S315080044F0FFF7A2FC03E0002038BD002038BD2046A7
S3150800450038BD00BF2DE9F04106460C4617461D4644
S315080045104FEA51284FEA48280368B3F1FF3F06D10E
S3150800452040F8048B41464FF40072FFF785FC336868
S31508004530434505D030464146FFF7B2FF0646D0B19F
S315080045403368E41A3444043408F50078FEF7DEFFCD
S31508004550331DE31AB3F5007F06D330464146FFF70D
S315080045609FFF064650B1041D17F8013B04F8013BAE
S31508004570013DEBD105E00020BDE8F0810020BDE853
S31508004580F0810120BDE8F08140F65453C2F20003E1
S315080045904FF0FF321A6040F65033C2F200031A6039
S315080045A0704700BF70B504460D461646FFF7EEFE87
S315080045B0FF281BD0681E2044FFF7E8FEFF2817D007
S315080045C0620A4FF4C043C0F60003B3EB422F07BF9D
S315080045D040F65030C2F2000040F65450C2F20000D5
S315080045E0214632462B46FFF78DFF70BD002070BD71
S315080045F0002070BD2DE9F84304460E46FFF7C6FEB7
S315080046000546701E2044FFF7C1FE0446FF2D18BF5D
S31508004610FF2800F0AB80854200F29F80022D40F211
S315080046209F800F2800F29F804FF40053C4F20203C4
S3150800463040F22312C4F267525A6048F6AB12CCF61F
S31508004640EF525A603422DA60DB6813F0010F04D0A7
S31508004650FFF792FE0020BDE8F8834FF40053C4F23A
S3150800466002031A6942F002021A6145F27809C0F695
S3150800467000094F460026FEF749FF3B7AAB4208D1B0
S3150800468045F27803C0F6000306EB460253F822709B
S3150800469005E001360C370D2EEDD14FF0FF37C84631
S315080046A00025FEF733FF98F80830A34208D145F2F3
S315080046B07803C0F6000305EB450253F8228006E0AE
S315080046C0013508F10C080D2DEBD14FF0FF384E4699
S315080046D00025FEF71BFF337AA34209D145F278037A
S315080046E0C0F6000305EB450203EB82035B6804E0B2
S315080046F001350C360D2DECD10023C7EB08084344D1
S31508004700C3F38F23E3B1013B9EB20136B6020025FF
S315080047104FF40054C4F20204EB196361236943F0B1
S3150800472040032361E36813F0010F05D0FEF7EEFEA0
S31508004730E36813F0010FF9D105F58065B542EBD1B1
S315080047404FF40053C4F202031A6922F002021A61F6
S31508004750FFF712FE0120BDE8F8830020BDE8F883C4
S315080047600020BDE8F8830020BDE8F8830020BDE8F6
S31508004770F88300BF00B583B040F65033C2F2000399
S315080047801B68B3F1FF3F08BF01201CD040F6503329
S31508004790C2F2000399685A681144DA6811441A6922
S315080047A011445A6911449A690A44D96953185B42F3
S315080047B002AA42F8043D46F25010C0F60000042151
S315080047C0FFF7F0FEFFE703B05DF804FB46F20402CC
S315080047D0C0F600024FF4C043C0F6000310681B6819
S315080047E0184446F20803C0F600031B68184446F24C
S315080047F00C03C0F600031B68184446F21003C0F603
S3150800480000031B68184446F21403C0F600031B682D
S31508004810184446F21803C0F600031B68184446F20B
S315080048205013C0F600031B681844D0F1010038BFC6
S315080048300020704708B540F65033C2F200031B68E3
S31508004840B3F1FF3F06D040F65030C2F20000FFF742
S31508004850BFFD88B140F65453C2F200031B68B3F19A
S31508004860FF3F0BD040F65450C2F20000FFF7B0FDF0
S31508004870003018BF012008BD002008BD012008BD72
S315080048804FF4C040C0F60000704700BF08B545F2B7
S315080048901410C0F600003121FFF7ACFA08BD00BFBE
S315080048A072B6704762B6704710B515498D4640F224
S315080048B00002C2F2000240F20803C2F200039A4262
S315080048C010D2131D0D4CE41A24F0030404340023FB
S315080048D0104645F24821C0F600015A581A500433CA
S315080048E0A342FAD1074808494FF000028842B8BFE8
S315080048F040F8042BFADBFBF7D3FC10BD0B000020B5
S315080049005811002008000020580F00208307F0B433
S3150800491048D0541E002A43D0CDB2034602E0002CEC
S315080049203ED0144603F8015B13F0030F04F1FF327F
S31508004930F5D1032C2DD9CDB20F2C45EA052545EA2C
S31508004940054518D9A4F1100703F110061A463F09C0
S3150800495006EB07161560103242F80C5C42F8085C44
S3150800496042F8045CB242F5D104F00F040137032C77
S3150800497003EB07130DD91E462246043A46F8045B94
S31508004980032AFAD8221F04F0030422F00302043291
S3150800499013442CB1C9B21C4403F8011BA342FBD132
S315080049A0F0BC704714460346C3E700BF2F64656D25
S315080049B06F70726F675F6F6C696D65785F73746D22
S315080049C03332703130332E73726563002F626F6F26
S315080049D0746C6F672E747874000000006D61696EE0
S315080049E02E630000222A3A3C3E3F7C7F00000000EE
S315080049F02B2C3B3D5B5D0000809A45418E418F80A4
S31508004A004545454949498E8F9092924F994F55553C
S31508004A1059999A9B9C9D9E9F41494F55A5A5A6A726
S31508004A20A8A9AAABACADAEAFB0B1B2B3B4B5B6B780
S31508004A30B8B9BABBBCBDBEBFC0C1C2C3C4C5C6C770
S31508004A40C8C9CACBCCCDCECFD0D1D2D3D4D5D6D760
S31508004A50D8D9DADBDCDDDEDFE0E1E2E3E4E5E6E750
S31508004A60E8E9EAEBECEDEEEFF0F1F2F3F4F5F6F740
S31508004A70F8F9FAFBFCFDFEFF01030507090E101203
S31508004A801416181C1E0000007D1D0100632C001E54
S31508004A909601A01E5A01001F0806101F0606201FB1
S31508004AA00806301F0806401F0606511F0700591F33
S31508004AB0521F5B1F541F5D1F561F5F1F601F08068E
S31508004AC0701F0E00BA1FBB1FC81FC91FCA1FCB1FE6
S31508004AD0DA1FDB1FF81FF91FEA1FEB1FFA1FFB1F60
S31508004AE0801F0806901F0806A01F0806B01F0400AE
S31508004AF0B81FB91FB21FBC1FCC1F0100C31FD01F90
S31508004B000206E01F0206E51F0100EC1FF21F010066
S31508004B10FC1F4E2101003221702110028421010060
S31508004B208321D0241A05302C2F04602C0201672C0F
S31508004B300601752C0201802C6401002D260841FF10
S31508004B401A030000C700FC00E900E200E400E000E8
S31508004B50E500E700EA00EB00E800EF00EE00EC00F5
S31508004B60C400C500C900E600C600F400F600F2005D
S31508004B70FB00F900FF00D600DC00A200A300A50098
S31508004B80A7209201E100ED00F300FA00F100D10040
S31508004B90AA00BA00BF001023AC00BD00BC00A100EB
S31508004BA0AB00BB0091259225932502252425612576
S31508004BB06225562555256325512557255D255C25EE
S31508004BC05B251025142534252C251C2500253C2578
S31508004BD05E255F255A2554256925662560255025B5
S31508004BE06C25672568256425652559255825522588
S31508004BF053256B256A2518250C25882584258C259B
S31508004C0090258025B103DF009303C003A303C303E4
S31508004C10B500C403A6039803A903B4031E22C6035A
S31508004C20B50329226122B1006522642220232123AB
S31508004C30F7004822B0001922B7001A227F20B200D6
S31508004C40A025A00061001A03E0001703F800070377
S31508004C50FF00010078010001300132010601390127
S31508004C6010014A012E017901060180014D00430217
S31508004C7081018201820184018401860187018701FD
S31508004C8089018A018B018B018D018E018F019001AB
S31508004C909101910193019401F601960197019801FA
S31508004CA098013D029B019C019D0120029F01A001E4
S31508004CB0A001A201A201A401A401A601A701A701BE
S31508004CC0A901AA01AB01AC01AC01AE01AF01AF016C
S31508004CD0B101B201B301B301B501B501B701B8011C
S31508004CE0B801BA01BB01BC01BC01BE01F701C00194
S31508004CF0C101C201C301C401C501C401C701C8017C
S31508004D00C701CA01CB01CA01CD011001DD010100AD
S31508004D108E01DE011201F3010300F101F401F40131
S31508004D20F8012801220212013A020900652C3B0209
S31508004D303B023D02662C3F02400241024102460206
S31508004D400A015302400081018601550289018A0140
S31508004D5058028F015A0290015C025D025E025F02F0
S31508004D6093016102620294016402650266026702A7
S31508004D70970196016A02622C6C026D026E029C0112
S31508004D80700271029D01730274029F017602770216
S31508004D90780279027A027B027C02642C7E027F0208
S31508004DA0A60181028202A90184028502860287027F
S31508004DB0AE014402B101B20145028D028E028F0294
S31508004DC090029102B7017B030300FD03FE03FF0374
S31508004DD0AC0304008603880389038A03B10311031D
S31508004DE0C2030200A303A303C4030803CC030300FE
S31508004DF08C038E038F03D8031801F2030A00F90304
S31508004E00F303F403F503F603F703F703F903FA03C9
S31508004E10FA033004200350041007600422018A04B0
S31508004E203601C1040E01CF040100C004D0044401B8
S31508004E3061052604000000004F70656E424C540060
S31508004E40303A00002E2E2F2E2E2F2E2E2F536F7512
S31508004E507263652F66696C652E6300004669726D1C
S31508004E607761726520757064617465207265717505
S31508004E706573742064657465637465640A0D00005F
S31508004E804F70656E696E67206669726D77617265C7
S31508004E902066696C6520666F722072656164696E4A
S31508004EA0672E2E2E000000004552524F520A0D0062
S31508004EB04F4B0A0D000000005374617274696E67E7
S31508004EC0207468652070726F6772616D6D696E67B0
S31508004ED02073657175656E63650A0D00506172739E
S31508004EE0696E67206669726D776172652066696C9E
S31508004EF06520746F206465746563742065726173D8
S31508004F006520626C6F636B732E2E2E00457261737B
S31508004F10696E672000000000206279746573206658
S31508004F20726F6D206D656D6F7279206174203078AF
S31508004F300000000052656164696E67206C696E65E1
S31508004F402066726F6D2066696C652E2E2E4552524C
S31508004F504F520A0D00000000496E76616C696420A4
S31508004F60636865636B73756D20666F756E642E2E48
S31508004F702E4552524F520A0D0000000050726F67BC
S31508004F8072616D6D696E6720000000002062797499
S31508004F90657320746F206D656D6F7279206174205A
S31508004FA03078000057726974696E672070726F678F
S31508004FB072616D20636865636B73756D2E2E2E00A6
S31508004FC0436C6F73696E67206669726D7761726587
S31508004FD02066696C650A0D004669726D77617265AF
S31508004FE02075706461746520737563636573736691
S31508004FF0756C6C7920636F6D706C657465640A0DE9
S31508005000000000002E2E2F2E2E2F2E2E2F536F75BA
S315080050107263652F41524D434D335F53544D3332BE
S3150800502046312F63616E2E630000000005020602FA
S31508005030060307030803090309040A040B040C04FE
S315080050400C050D050E050F050F06100610071008AE
S315080050502E2E2F2E2E2F2E2E2F536F757263652F01
S3150800506041524D434D335F53544D333246312F75BC
S315080050706172742E630000000060000800200000C2
S315080050800300000000800008002000000400000063
S3150800509000A00008002000000500000000C000086D
S315080050A0002000000600000000E0000800200000C4
S315080050B007000000000001080020000008000000AA
S315080050C00020010800200000090000000040010837
S315080050D0002000000A00000000600108002000000F
S315080050E00B00000000800108002000000C000000F2
S315080050F000A00108002000000D00000000C0010803
S31508005100002000000E00000000E00108002000005A
S315080051100F0000002E2E2F2E2E2F2E2E2F536F759A
S315080051207263652F41524D434D335F53544D3332AD
S3150800513046312F4743432F766563746F72732E6328
S3150800514000000000002020202020202020202828E1
S315080051502828282020202020202020202020202029
S315080051602020202020881010101010101010101069
S315080051701010101010040404040404040404041099
S315080051801010101010104141414141410101010127
S3150800519001010101010101010101010101010101F1
S315080051A010101010101042424242424202020202FD
S315080051B002020202020202020202020202020202C1
S315080051C01010101020000000000000000000000071
S315080051D000000000000000000000000000000000C1
S315080051E000000000000000000000000000000000B1
S315080051F000000000000000000000000000000000A1
S315080052000000000000000000000000000000000090
S315080052100000000000000000000000000000000080
S315080052200000000000000000000000000000000070
S315080052300000000000000000000000000000000060
S30D08005240000000000000000058
S30D080052480104000044510008AE
S70508000000F2
